:06000000803169290000B7
:0800080083018A012000770842
:10001000A0007808A1007908A2007A08A300850151
:1000200091308400801D162891191F282008F700A0
:100030002108F8002208F9002308FA00090080319D
:1000400032282400110820003608240091001516DB
:1000500020009111240014182B28F801151AF80A11
:10006000200008002400941A3D282000AD0124003F
:10007000141D3D282000AD17240020002D08AD0AD6
:10008000B30033087F3C031858283308803C031D15
:1000900051282B08B400B501B5012B08B60021206A
:1000A00057282A08B400B5012A08B60021201B29C8
:1000B000B30803191129240015132000911D5E288F
:1000C0002400110815162000B100310803198D28ED
:1000D000013A03199828033A0319B628013A03197B
:1000E000BB28133A0319C028013A0319C028033A60
:1000F0000319C028013A0319C028333A0319FB2811
:10010000103A0319FF28013A03190329033A031986
:100110000729013A03190B290F299701013096008D
:10012000AC00A501A401A701A601A901A8011029FD
:10013000AC080319B4281708FA001608F7001708C6
:100140007A02031D9B287708A8007A08A9002908CD
:100150002502031CB428031DB12824082802031813
:10016000B428A60A0319A70AAC0110292708AB0076
:100170002608AA0010292908AB002808AA0010297F
:1001800010303102B400340DF700F70DFC30F705E4
:1001900021001D08C33977049D009D1420003410F0
:1001A00021009D18D6282000341421002000341886
:1001B000E228341021009D18E0282000341421008A
:1001C000D628200021009D18E3281C08FA001B08EF
:1001D0002000B5007A08B6003508F8003608F900A6
:1001E0007908AB007808AA00AA0DAB0DAA0DAB0DDB
:1001F000FC30AA051029AB010D08AA001029220025
:100200000D102000102922000D14200010292200BA
:100210008D102000102922008D1420001029102993
:100220001B29240015132000911D142924001108F6
:1002300015162000B200911180311628FF302100E0
:100240008C008D008E0022009D12853020009800C9
:1002500099019701960121001E169E161E139E17E6
:100260001D141E109E101E110D3023008C00003036
:1002700090008D008F00F80021001D08C33978041C
:100280009D00FC3024008D00210095130D102200EC
:100290000D1421008D1022008D1421000E168E15D4
:1002A0008031200090292030850010308400000823
:1002B000031967290A30F800F701F70B5D29F80BDD
:1002C0005C295F30F700F70B6329800B5A298031D6
:1002D000CA29850184011F30830521008E150E1661
:1002E000A0302400920036309500F43021009900AF
:1002F00001302000AC000330AD002F0091019201CD
:10030000980199019A0123008C018D01220092012C
:10031000910194019301F0302100990020001E29E1
:100320000130AC00A901A8012908A7002808A600EF
:100330002708A5002608A400970196012100911521
:10034000C0308B042000AC080319CA291708FA0032
:100350001608F70017087A02031DA6297708AE00D1
:100360007A08AF002F082502031CBF29031DBC29F2
:1003700024082E020318BF29A60A0319A70A2F086A
:10038000A9002E08A8002908A5002808A40001300B
:08039000B0005329A32963000A
:020000040001F9
:04000E008439FF1E14
:00000001FF
